:020000020000FC
:0200000007C037
:02000A0088C1AB
:10000E008EC10FED0DBF01E809B900E007BB0FEF80
:10001E0008BB00E001BB01E002BB539A549A579A09
:10002E00FBD0FFD012D071E0789452C00F9303E74B
:10003E00EFD00F910895482C372C262C2A94F1F7E7
:10004E003A94D9F74A94C1F7089504E6602E00E079
:10005E00702E0FEF802EEFDF0FE8602E0AEF702E5E
:10006E0002E0802EE8DF08957F7700E00FBD00E00C
:10007E000DBD0CBDEE27FF2700E809BF07E00EBD42
:10008E00E4DF9A94E9F700E00EBD09BF089501E39D
:10009E00BFD0CCDFC1D001E0902EE6DF4CD018C02F
:1000AE0001E3B6D000E3B4D0C1DFB6D00AE0902EA3
:1000BE00DBDF41D00DC001E3ABD000E3A9D000E3FC
:1000CE00A7D0B4DFA9D004E6902ECEDF34D000C086
:1000DE00072F07700130D9F2023011F3033059F3B4
:1000EE00043081F0F5CF02E8602E0EEF702E0AE09C
:1000FE00802EA1DF01E0602E01E0702E0EEB802E2F
:10010E009ADF08957F7600E00FBD00E00DBD0CBDB7
:10011E00EE27FF2700E809BF07E00EBD74FD07C0FC
:10012E000AD0E1DFE0DFDFDFDEDFDDDFF7CF00E08B
:10013E000EBD09BFCDCFAA277F7B2CB53DB54E2F67
:10014E005F2F8CD0062F0CD0052F0AD0042F08D08D
:10015E00032F06D0022F04D077FD7BD05DD00895FB
:10016E000F9302950F70006339D00F910F700063DB
:10017E0035D008950F93072F0770043009F401E06E
:10018E0002950A2B0230E1F00530D1F00830C1F0B3
:10019E000131B1F00431A1F0073191F0033281F059
:1001AE00063271F0023361F0053351F00A3161F01D
:1001BE00093251F0083341F00A3051F00F91089591
:1001CE000CE226D00F9108950EE222D00F910895E1
:1001DE0000E31ED00EE21CD00F910895A395B72F09
:1001EE00B770B295BA2BB93209F47064B83309F40A
:1001FE007064003321F070640BD0BCDF089576FF7D
:10020E0003C006D0B7DF0895AA3011F000E200C097
:10021E005D9BFECF0CB908950AE0FADF0DE0F8DF22
:10022E000895EF93FF93F2E0E0E40BD0FF91EF918E
:10023E0008956E666D7472303430393136410A0D60
:10024E000000C895002021F0002DE2DF3196F9CF95
:10025E0008950F930BE2DCDF0F9108950F931F9318
:10026E007F938F932FD0242F352F462F572F682F04
:10027E008F917F911F910F9108958F937F936F931D
:10028E005F934F932F913F914F915F916F918F910C
:10029E007F911F910F910895042F152F6FEF639586
:1002AE0000511742E0F75FE9505108511C4FE0F33F
:1002BE00539504561040E0F740EA4051065FE8F3CC
:1002CE00400F0895E9DF77278EEF4D5C43FF4350D3
:1002DE0047FF40535D5C53FF535057FF50536D5CC7
:1002EE0063FF635067FF6053220F331F441F551F78
:1002FE00661F771F881F4AF3111F18F77D5C73FF67
:10030E00735077FF70538D5F83FF8350DECF0F9353
:10031E000FB7319609F470680FBF0F9118950F93B0
:10032E000FB70F930BB10CB10F7D023599F0072F5C
:10033E0007700395053061F0787F702B706101E0D6
:10034E00902E602E702E802E0F910FBF0F9118954C
:10035E0001E0F2CF072F0770043049F700E00DBD22
:08036E000CBDEE27FF27F0CFC4
:00000001FF
